:030000000297E381
:03000300021312D3
:03000B00020BB530
:0300330002081CA4
:03004300020A00AE
:03005B0002833BE2
:10037000907FE9E070030204731470030204E72421
:10038000FE700302054F24FB700302046414700323
:1003900002045214700302043A1470030204492444
:1003A00005600302059E907FEBE024FE601614605A
:1003B000362402707B7412907FD4F07400907FD545
:1003C000F00205A5907FEAE0FF120A99EA49600D64
:1003D000EA907FD4F0E9907FD5F00205A5907FB434
:1003E000E04401F00205A5907FEAE0FF120A58EA16
:1003F00049603312A23BF54E907FEEE0FFE54ED30D
:100400009F4003E0F54EE54ED394404003754E40C7
:10041000AE02AF017C7F7D00AB4E129137907FB56D
:10042000E54EF00205A5907FB4E04401F00205A579
:10043000907FB4E04401F00205A5907F00E521F033
:10044000907FB57401F00205A5907FEAE0F52102E6
:1004500005A5907FEAE0F535D202438810D2EBD2B1
:10046000A80205A5907F00E535F0907FB57401F0F6
:100470000205A5907FE8E0247F6024146031240207
:10048000705BA200E433FF25E0FFA205E4334F9048
:100490007F00F0E4A3F0907FB57402F00205A5E4BC
:1004A000907F00F0A3F0907FB57402F00205A59054
:1004B0007FECE0F45480FFC4540FFFE054072F2575
:1004C000E024B4F582E4347FF583E05401907F00AA
:1004D000F0E4A3F0907FB57402F00205A5907FB41C
:1004E000E04401F00205A5907FE8E024FE601D24B1
:1004F0000260030205A5907FEAE0B40105C2000294
:1005000005A5907FB4E04401F00205A5907FEAE0E4
:100510007034907FECE0FF5407FEF54EEF30E703B8
:10052000434E10907FD7E54EF0E54E4420F0EFF4B7
:100530005480FDC4540F2E25E024B4F582E4347FAA
:10054000F583E4F0805F907FB4E04401F080569042
:100550007FE8E024FE60182402704A907FEAE0B44D
:100560000104D200803F907FB4E04401F0803690D7
:100570007FEAE07020907FECE0F45480FFC4540FD9
:10058000FFE054072F25E024B4F582E4347FF5839F
:100590007401F08010907FB4E04401F08007907FF8
:0C05A000B4E04401F0907FB4E04402F0AD
:0105AC00222C
:1005AD00754AFF7549FF75480F754700D203C2069E
:1005BD00C202C200C205C2019003007419F0E4909A
:1005CD0001BCF0C2049001C0F0A3F0C2AFC2A812EA
:1005DD000C22E49002AFF09001BDF0900100F0A369
:1005ED00F0A3F0A3F0A3F0A37410F0A37401F0A393
:1005FD007408F07E017F001219C1754C12754D0AF9
:10060D0090010BE0FF054DE54DAC4C7002054C140F
:10061D00F5828C83EFF090010CE04480FF054DE5F1
:10062D004DAC4C7002054C14F5828C83EFF09001AB
:10063D000DE0FF054DE54DAC4C7002054C14F582F7
:10064D008C83EFF090010EE0FF054DE54DAC4C7045
:10065D0002054C14F5828C83EFF090120AE493FF9F
:10066D0074019390011CCFF0A3EFF090011CE0FFFB
:10067D00A3E0FEEF6EFF90011CF0A3E06FFFF09082
:10068D00011CE06FF0E0FEA3E0FFE4FCFD755210ED
:10069D007553027554127555AC129426754C12751E
:1006AD004DB290010DE0FF054DE54DAC4C700205CE
:1006BD004C14F5828C83EFF090010EE0FF054DE5B3
:1006CD004DAC4C7002054C14F5828C83EFF0907F8D
:1006DD0092E0FFC4540F2441FF054DE54DAC4C7025
:1006ED0002054C14F5828C83EFF0054DE54DAE4CB3
:1006FD007002054C14F5828E83E4F07582107583BB
:10070D0001E0FCA3E0FDA3E0FEA3E0FF90011812C1
:10071D00A3EE7E017F181286BE900118E0FCA3E0C7
:10072D00FDA3E0FEA3E0FF75520A75530675541242
:10073D007555B8129426D2E843D820907FAB74FF3C
:10074D00F05391EF907FAFE04401F0907FAEE04425
:10075D001FF0D2AF20012E20012BA2039207120908
:10076D00C575465075456D7544337543002001E4DC
:10077D007FFF7EFF7DFF7CFF784312A3D7EC4D4EAC
:10078D004F60D180E8300105120370C20130060AB6
:10079D001209FB5003120AE8C20612965E9001BDC3
:1007AD00E0600C129201E49001BDF0907FD3F090C7
:1007BD0002AFE0B40F031299B912A095E4FF7401D2
:1007CD00A807088002C333D8FCFE9001BCE05E6030
:1007DD001474282FF8E6D3940A40047E0180027E1B
:1007ED00008E4B8003754B0174682FF582E4342025
:1007FD00F583E54BF00FBF04C5E52CD3940A4004F7
:0E080D007F0180027F0090206CEFF0020792C6
:01081B0022BA
:04081C0053D8EF328C
:10082000E533C39401400E907F93E04430F0907F15
:1008300095E044C0F07FF47E011209AE907F96E00F
:1008400054FEF07F0A7E001209AE907F96E04408C5
:10085000F07F057E001209AE907F96E054FBF07F9A
:10086000057E001209AEE533C39401500E7F027D70
:10087000FF1282EA7F057E001209AE907F96E04467
:1008800002F0E0547FF07F057E001209AE907F9663
:10089000E04440F07F057E001209AE907F96E05460
:1008A000BFF07F327E001209AE907F96E04440F0A8
:0808B0007F327E001209AE2226
:1008B800907F96E054FDF0E04480F07F0A7E0012BD
:1008C80009AEE533C39401500E7F02E4FD1282EABB
:1008D8007F057E001209AE907F96E054BFF07F0539
:1008E8007E001209AE907F96E04404F07F057E00FA
:1008F8001209AE907F96E054F7F07F057E0012094A
:10090800AE907F96E04401F07F057E001209AEE5C7
:1009180033C39401400E907F93E054CFF0907F95BD
:08092800E0543FF0120B002225
:10093000900AF4E4937076907F937430F0907F94F3
:10094000743CF0907F9574C6F07F0A7E001209AE69
:10095000E4907F9CF0907F967408F0907F9C74CF19
:10096000F07F0A7E001209AE902070E0FFC4540FA1
:10097000F533C394015007907F96E04480F0E490F3
:100980007F97F0907F9D7402F0E533C39401400B94
:10099000E4907F98F0907F9E74C0F0907FE2741294
:0E09A000F01208207582F475830A74FFF022AD
:1009AE008E5D8F5EE55E155EAE5D7002155D4E600E
:0709BE00051209EA80EE2298
:1009C500907FD6E054FBF0E04408F0300704E044A3
:1009D50002F07FD07E071209AE907FD6E054F7F083
:0509E500E04404F022D3
:1009EA007400F58690FDA57C05A3E582458370F920
:0109FA0022DA
:0509FB001208B8D32230
:100A0000020C4E00020C8100020C6600020CC000B9
:100A1000020CAA00020AED00020AEE00020AEF0030
:100A2000020CDB00020DCB00020D1700020E2B00A2
:100A3000020D5300020E8B00020D8F00020EEB0020
:100A4000020AF000020AF200020AF100020AF300B0
:080A5000020F4B00020F6100D0
:020A58008F4FBE
:100A5A00E4F5507551FF75521275536AAB51AA529B
:100A6A00A95390000112A254B4031DAF500550EFD0
:100A7A00B54F012212A23B7E0029FFEE3AA9077563
:0E0A8A0051FFF552895380D47B007A00790029
:010A9800223B
:100A9900E4FE7551FF755212755312AB51AA52A952
:100AA9005390000112A2546402702DAD060EEDB5EB
:100AB90007012290000212A2AD85F04FF550624F56
:100AC900E54F6250E550624F29FDE54F3AA905759A
:0E0AD90051FFF552895380C37B007A007900EB
:010AE70022EC
:050AE800120820D322DA
:010AED0032D6
:010AEE0032D5
:010AEF0032D4
:010AF00032D3
:010AF10032D2
:010AF20032D1
:010AF30032D0
:030AF400000407F4
:090B0000907FD6E04480F080747F
:100B7D00438701000000000000000000000000227B
:100B8D00538EF7E58954F14401F589758CB1D2A9DD
:100B9D0075984075CBFF75CAF375C834E4FF7F05B2
:070BAD007828E4F608DFFCE4
:010BB400221E
:100BB500C0E0C083C082C0D075D000C000C006C0F0
:010BC5000728
:100BC600300416758CF8758A307F2FAE071FEE60DD
:100BD6003C9020007455F080F2758CB17F28EFD3DD
:100BE600942C5009A807E66001160F80F1900300C7
:100BF600E0600214F09001C0E07002A3E0600E9085
:0D0C060001C1E024FFF09001C0E034FFF0D8
:0F0C1300D007D006D000D0D0D082D083D0E0322E
:100C2200D200758E10120930E533C394014008904A
:100C32007F927402F08005E4907F92F0128000129D
:0C0C42000F7D1294F7121B0C120B8D2278
:100C4E00C0E0C083C082D2015391EF907FAB74019C
:080C5E00F0D082D083D0E03217
:100C6600C0E0C083C082907FC4E4F05391EF907FD0
:0B0C7600AB7404F0D082D083D0E032D9
:100C8100C0E0C083C0825391EF907FAB7402F090BB
:100C91007FD8E0700D907FD9E07007E52C70037567
:090CA1002C14D082D083D0E03283
:100CAA00C0E0C083C0825391EF907FAB7410F0D044
:060CBA0082D083D0E0327D
:100CC000C0E0C083C082300202D2065391EF907F11
:0B0CD000AB7408F0D082D083D0E0327B
:100CDB00C0E0C083C082C0D075D0105391EF907F1D
:100CEB00A97402F0E53430E013E53230E0079020D0
:100CFB0004E04401F0902001E04401F0E52C700386
:0C0D0B00752C14D0D0D082D083D0E03200
:100D1700C0E0C083C082C0D075D0105391EF907FE0
:100D2700A97404F0E53430E113E53230E10790208F
:100D37000CE04401F0902009E04401F0E52C700339
:0C0D4700752C14D0D0D082D083D0E032C4
:100D5300C0E0C083C082C0D075D0105391EF907FA4
:100D6300A97408F0E53430E213E53230E20790204D
:100D730014E04401F0902011E04401F0E52C7003ED
:0C0D8300752C14D0D0D082D083D0E03288
:100D8F00C0E0C083C082C0D075D0105391EF907F68
:100D9F00A97410F0E53430E313E53230E307902007
:100DAF001CE04401F0902019E04401F0E52C7003A1
:0C0DBF00752C14D0D0D082D083D0E0324C
:100DCB00C0E0C083C082C085C084C086758600C069
:100DDB00D075D0105391EF907FAA7402F0E53420B8
:100DEB00E006907FC7F08022E53130E00A907FC7A4
:100DFB00E09002F8F08013E52230E007902004E049
:100E0B004402F0902001E04402F0E52C7003752CB5
:100E1B0014D0D0D086D084D085D082D083D0E0328D
:100E2B00C0E0C083C082C085C084C086758600C008
:100E3B00D075D0105391EF907FAA7404F0E5342055
:100E4B00E106907FC9F08022E53130E10A907FC93D
:100E5B00E09002F9F08013E52230E10790200CE0DE
:100E6B004402F0902009E04402F0E52C7003752C4D
:100E7B0014D0D0D086D084D085D082D083D0E0322D
:100E8B00C0E0C083C082C085C084C086758600C0A8
:100E9B00D075D0105391EF907FAA7408F0E53420F1
:100EAB00E206907FCBF08022E53130E20A907FCBD7
:100EBB00E09002FAF08013E52230E207902014E074
:100ECB004402F0902011E04402F0E52C7003752CE5
:100EDB0014D0D0D086D084D085D082D083D0E032CD
:100EEB00C0E0C083C082C085C084C086758600C048
:100EFB00D075D0105391EF907FAA7410F0E5342089
:100F0B00E306907FCDF08022E53130E30A907FCD70
:100F1B00E09002FBF08013E52230E30790201CE009
:100F2B004402F0902019E04402F0E52C7003752C7C
:100F3B0014D0D0D086D084D085D082D083D0E0326C
:100F4B00C0E0C083C0825391EF907FA97480F0D032
:060F5B0082D083D0E032D9
:100F6100C0E0C083C0825391EF907FAA7480F0905B
:0C0F710001BD74FFF0D082D083D0E032CC
:100F7D0090012012A3FA000025809001247408F03E
:100F8D00A37401F0A3746EF0A3F0A37413F0A37413
:100F9D0011F0E4A3F0A3F090011EF090011EE0FF0C
:100FAD0004A3F0EF75F00DA42401F9740335F0A836
:100FBD0001FC7D017B017A01791F7E007F0D12A25C
:100FCD00127E017F1F1287A690011EE004F0E0C380
:100FDD00940440C7E4F52790011EF090011EE0FF38
:100FED00C39404501A74F82FF582E43402F583E4A7
:100FFD00F074232FF8E4F690011EE004F080DCE499
:10100D00F534E5C0602F90011E7401F090011EE0D3
:10101D00FFD39404501FEF14FF7401A8070880023A
:10102D00C333D8FC42347E017F1E12844190011ED1
:10103D00E004F080D7E4F53EF522F531F53290016C
:10104D001EF090011EE0FF75F008A42406F582E461
:10105D003420F583E054F0FE74C52FF582E434019D
:10106D00F583EEF0743A2FF8A60674362FF8E4F6F1
:10107D00742D2FF8E4F674FC2FF582E43402F58319
:10108D00E4F090011EE004F0E0B404B6902060E0BE
:04109D00540FF54EA9
:1010A1007003021126E490011EF090011EE0FFC3BF
:1010B100940450E47401A807088002C333D8FC5596
:1010C1004E605A90011EE0FE75F008A42402F582DC
:1010D100E43420F583E0FFEE75F008A42405F582E1
:1010E100E43420F583E0EE75F008A42406F582E4EB
:1010F1003420F583E0FFAF06EE75F00DA42402F570
:1011010082E43403F583E0FCA3E0FDA3E0FEA3E069
:10111100F5668E658D648C637D061283DF90011EFA
:06112100E004F0808522CD
:02112700AC0713
:10112900907FA5E04480F0EC25E04441907FA6F053
:101139007B3CAF031BEF7016907FA5E04440F09015
:101149007FA6E0FD7D32AF051DEF60D480F8907F6A
:10115900A5E0FD30E0DC20E109E04440F07EFF7FBE
:10116900F922ED30E20C907FA5E04440F07EFF7F4C
:10117900FA22907FA5E04420F0907FA6E0FD7B1E37
:10118900AF031BEF7016907FA5E04440F0907FA657
:10119900E0FD7D32AF051DEF608680F8907FA5E008
:1011A900FD20E0DC7B3CAF031BEF7019907FA5E0CD
:1011B9004440F0907FA6E0FD7D32AF051DEF70033E
:1011C90002112980F5907FA5E0FD30E0D930E209D0
:1011D900E04440F07EFF7FFA22C2AF907FA5E04451
:0C11E90040F0907FA6E0FDD2AFFF7E003A
:0111F50022D7
:1012000012010001FFFFFF401007018042000102B0
:10121000030109025800010104803C090400000A8E
:10122000FFFFFF050705810240000007050102409E
:10123000000007058202400000070502024000008E
:101240000705830240000007050302400000070570
:1012500084024000000705040240000007058702E1
:1012600040000007050702400000040309042403AE
:1012700043006F006E006E00650063007400200084
:101280005400650063006800200049006E006300A0
:101290002E001803570068006900740065004800BC
:1012A0004500410054002D0034001A035800580036
:1012B0002D00580058002D005800580058005800C4
:1012C000580058002A0343006F006E006600690052
:1012D0006700750072006100740069006F006E00A5
:1012E000200053007400720069006E006700220342
:1012F00049006E00740065007200660061006300C2
:101300006500200053007400720069006E006700E1
:021310000000DB
:10131200C0E0C0F0C083C082C085C084C086C0D097
:1013220075860075D018902060E0540FF5F07011AA
:10133200D0D0D086D084D085D082D083D0F0D0E0F7
:101342003275860010F00B10F11210F21910F32012
:1013520080D4E528700375281402137CE5297003F4
:1013620075291402150DE52A7003752A1402169EBA
:10137200E52B7003752B1402182F902002E0543FC6
:1013820020E23A20E10B20E40B20E514600902136D
:1013920043021465021343438204E0F53A02134305
:1013A200438204E0432D010213435382F843820532
:1013B200E042365382FBE054FBF002134330E10279
:1013C20080E8F585E53230E00A5382F8438204E092
:1013D20054FEF0E58520E3569020507400F09020F2
:1013E200587401F0907FE2E04440F0907FE305867C
:1013F200907E800586E585F0A3E584F00586907FE2
:10140200E5E53FFD030303FEF0F0F0F0F0F0F0F04D
:10141200DEF6907FE2E054BFF09020587400F09026
:101422007FB7EDF0902001E054FEF00213437F40BD
:10143200907E800586902000E584FE2405FD8D8443
:10144200E08E8430E009E00586F0A30586DFEF0533
:1014520086C374409F907FB7F00586A3E054FEF0E8
:10146200021343532DFAE5236008752300D2E7FEE9
:10147200800A907FC7E0FE70030214FF9020507430
:1014820000F09020587401F0907FE2E04440F09028
:101492007FE30586907E400586E585F0A3E584F02E
:1014A2000586907FE5EE30E7080586E02438F005F2
:1014B20086EE547FFE5407FBEE547860300303033C
:1014C20030E30474077B08FDFCE0E0E0E0E0E0E0EC
:1014D200E0DDF6EBFE6019EC640770118B23907F60
:1014E200E2E054BFF09020587400F0801BE0DEFD73
:1014F200907FE2E054BFF09020587400F0902001F9
:10150200E054FDF0907FC7F002134390200AE054AC
:101512003F20E23A20E10B20E40B20E514600902AF
:1015220013430215F6021343438204E0F53B021310
:1015320043438204E0432E010213435382F8438261
:1015420005E042375382FBE054FBF002134330E1E3
:101552000280E8F585E53230E10A5382F8438204DD
:10156200E054FEF0E58520E3569020507401F0909F
:1015720020587401F0907FE2E04440F0907FE30550
:1015820086907E000586E585F0A3E584F0058690C9
:101592007FE5E540FD030303FEF0F0F0F0F0F0F02C
:1015A200F0DEF6907FE2E054BFF09020587400F035
:1015B200907FB9EDF0902009E054FEF00213437FD2
:1015C20040907E000586902008E584FE2405FD8D6E
:1015D20084E08E8430E009E00586F0A30586DFEF23
:1015E2000586C374409F907FB9F00586A3E054FE40
:1015F200F0021343532EFAE5246008752400D2E763
:10160200FE800A907FC9E0FE70030216909020507F
:101612007401F09020587401F0907FE2E04440F0B1
:10162200907FE30586907DC00586E585F0A3E5847D
:10163200F00586907FE5EE30E7080586E02438F075
:101642000586EE547FFE5407FBEE547860300303A8
:101652000330E30474077B08FDFCE0E0E0E0E0E037
:10166200E0E0DDF6EBFE6019EC640770118B24906C
:101672007FE2E054BFF09020587400F0801BE0DE5F
:0E168200FD907FE2E054BFF09020587400F01D
:10169000902009E054FDF0907FC9F00213439020A0
:1016A00012E0543F20E23A20E10B20E40B20E51445
:1016B0006009021343021787021343438204E0F5D3
:1016C0003C021343438204E0432F0102134353823D
:1016D000F8438205E042385382FBE054FBF00213EA
:1016E0004330E10280E8F585E53230E20A5382F8C2
:1016F000438204E054FEF0E58520E35690205074C8
:1017000002F09020587401F0907FE2E04440F090A5
:101710007FE30586907D800586E585F0A3E584F06E
:101720000586907FE5E541FD030303FEF0F0F0F050
:10173000F0F0F0F0DEF6907FE2E054BFF090205839
:101740007400F0907FBBEDF0902011E054FEF002A9
:1017500013437F40907D800586902010E584FE2411
:1017600005FD8D84E08E8430E009E00586F0A30558
:1017700086DFEF0586C374409F907FBBF00586A38C
:10178000E054FEF0021343532FFAE5256008752557
:1017900000D2E7FE800A907FCBE0FE7003021821A2
:1017A0009020507402F09020587401F0907FE2E095
:1017B0004440F0907FE30586907D400586E585F006
:1017C000A3E584F00586907FE5EE30E7080586E026
:1017D0002438F00586EE547FFE5407FBEE54786003
:1017E0003003030330E30474077B08FDFCE0E0E012
:1017F000E0E0E0E0E0DDF6EBFE6019EC640770117C
:101800008B25907FE2E054BFF09020587400F08068
:101810001BE0DEFD907FE2E054BFF09020587400A2
:10182000F0902011E054FDF0907FCBF00213439034
:10183000201AE0543F20E23A20E10B20E40B20E59F
:10184000146009021343021918021343438204E08F
:10185000F53D021343438204E04330010213435336
:1018600082F8438205E042395382FBE054FBF002E8
:10187000134330E10280E8F585E53230E30A538214
:10188000F8438204E054FEF0E58520E356902050B2
:101890007403F09020587401F0907FE2E04440F02F
:1018A000907FE30586907D000586E585F0A3E584BD
:1018B000F00586907FE5E542FD030303FEF0F0F0BE
:1018C000F0F0F0F0F0DEF6907FE2E054BFF0902010
:1018D000587400F0907FBDEDF0902019E054FEF0B8
:1018E0000213437F40907D000586902018E584FE1A
:1018F0002405FD8D84E08E8430E009E00586F0A3A8
:101900000586DFEF0586C374409F907FBDF0058696
:10191000A3E054FEF00213435330FAE52660087545
:101920002600D2E7FE800A907FCDE0FE7003021908
:10193000B29020507403F09020587401F0907FE230
:10194000E04440F0907FE30586907CC00586E58505
:10195000F0A3E584F00586907FE5EE30E708058684
:10196000E02438F00586EE547FFE5407FBEE5478F1
:10197000603003030330E30474077B08FDFCE0E000
:10198000E0E0E0E0E0E0DDF6EBFE6019EC6407701B
:10199000118B26907FE2E054BFF09020587400F045
:1019A000801BE0DEFD907FE2E054BFF09020587491
:1019B00000F0902019E054FDF0907FCDF002134329
:0119C00032F4
:0419C100AD07AC06BC
:1019C5007906ED2404F582E43CF583E0FAA3E0FB17
:1019D5004A7003021B09E9B407004003021ADB90B1
:1019E50019EBF8282873021AB9021A71021A5A0259
:1019F5001A40021A2F021A1A021A00907FA5E04413
:101A050080F08D828C83A3E0FF25E044A0907FA623
:101A1500F019021ADB198D828C83E0C39420400AE9
:101A2500A3A3E0907FA6F0021ADB8D828C83A3A38B
:101A3500E0A3E0907FA6F019021ADB907FA5E044B1
:101A450080F08D828C83A3E0FF25E044A1907FA6E2
:101A5500F019021ADBEB64014A7008907FA5E04497
:101A650020F019907FA6E0F55919806AED2404F558
:101A750082E43CF583E0FEA3E064024E7008907FAB
:101A8500A5E04420F019907FA6E0FFED2406F5823D
:101A9500E43CF583E475F00112A29785F082F583A5
:101AA500EFF0ED2404F582E43CF58374FFF5F012C4
:101AB500A2818022907FA5E04440F0907FA6E0FFC0
:101AC500ED2406F582E43CF583E0FAA3E0F5828A8D
:101AD50083EFF07F0822907FA5E0F55930E0F730DD
:101AE500E207E04440F07F0622E9D3940250030266
:101AF50019C7E55930E1030219C7907FA5E04440B5
:061B0500F07F07227F08BB
:011B0B0022B7
:101B0C00E533C39401501C7F057E001209AE7F02A1
:101B1C007DFF1282EA7F057E001209AE7F037DFFF6
:041B2C001282EA2215
:108000007BFF7A12791B90000412A254FD8B5075ED
:108010005112755224E4907FE1F0907FE0F0F54E2C
:10802000F54F9002AEF0907FDFF0907FDEF0907F12
:10803000A974FFF0907FAAF0E4FCEC25E024B4F5ED
:1080400082E4347FF583E4F00CBC10EEE4907FDD35
:10805000F0AF051DEF70030281C6AB50AA51A952C3
:1080600090000112A254640560030281B5900003E0
:1080700012A2546401600302813C90000212A254D7
:10808000FF547FFCD394075003028116ECC3941075
:108090004003028116EF30E742E54FAE4E7802CE44
:1080A000C313CE13D8F9FF74F02CF582E4347FF5B6
:1080B00083EFF0907FE0E0FFEC24F8FE7401A80667
:1080C000088002C333D8FC4F907FE0F09002AEE00E
:1080D00004F0907FDDE04480F0803EE54FAE4E78C6
:1080E00002CEC313CE13D8F9FF74E82CF582E43422
:1080F0007FF583EFF0907FE1E0FFEC24F8FE740160
:10810000A806088002C333D8FC4F907FE1F09002AC
:10811000AEE004F080037FFF2290000412A25425F9
:108120004FF54FE4354EF54E90000512A254FEE493
:10813000254FF54FEE354EF54E0281B8AB50AA51A2
:10814000A95290000312A254FF64026005EF640379
:10815000706090000212A254FF547FFCD394075029
:108160004EEF30E71E907FDEE0FF7401A804088028
:1081700002C333D8FCFE4F907FDEF0907FACE04E20
:10818000F08035907FDFE0FF7401A804088002C30F
:1081900033D8FCFE4F907FDFF0907FADE04EF0ECE7
:1081A00025E024C5F582E4347FF583ECF080097F77
:1081B000FF227FFF227FFF2274072552F552E4350C
:1081C00051F55102805120030D9002AEE0600790FE
:0881D0007FAEE04402F07F00E5
:0181D8002284
:0481D9008E598F5AD2
:1081DD00755B03E55A2404F582E43559F583E0FE19
:1081ED00A3E04E70030282E7E55B604E1460381425
:1081FD00602014600302828B907FA5E04480F0859F
:10820D005A82855983A3E0FF25E044A0907FA6F014
:10821D00806C855A82855983E0C394204009A3A3BD
:10822D00E0907FA6F08057155B855A82855983A310
:10823D00A3E0A3E0907FA6F08044E55A2406F582E2
:10824D00E43559F583E475F00112A29785F082F5B6
:10825D0083E0907FA6F0907FA5E04440F0E55A249E
:10826D0004F582E43559F58374FFF5F012A281858A
:10827D005A82855983A3A3E475F00112A281907FE0
:10828D00A5E0F55C30E0F730E207E04440F07F0612
:10829D0022E55C20E10A907FA5E04440F07F0722B3
:1082AD00E55B70317F017E001209AE907FA5E04441
:1082BD0080F0855A82855983A3E0FF25E044A09084
:1082CD007FA6F0907FA5E0F55C30E0F730E1D57545
:0C82DD005B030281E0155B0281E07F087A
:0182E9002272
:0282EA00AE07DD
:1082EC007C02EC14601514701E907FA5E04480F0A5
:1082FC00EE25E04440907FA6F0800C907FA6EDF038
:10830C00907FA5E04440F0907FA5E0FB30E0F8BC06
:10831C00020A20E107E04440F07F0722EB30E20A3A
:0E832C00907FA5E04440F07F0622DCB67F087B
:01833A002220
:10833B00C0E0C083C082C2A99003007419F0D2A917
:0F834B0053917F9001C4E4F0D082D083D0E03210
:10835A00EF75F008A42400F582E43420AB82FAF524
:10836A0083A3E4F08B828A83A3A3A3E0F56174BF9D
:10837A00F08B828A83A3A3E04410F08B828A83A3C2
:10838A00A3A3E4F08B828A83A3F0F9ED601D740144
:10839A007E00A807088005C333CE33CED8F9FFE4A0
:1083AA00EF5531600479098002790D8B828A83A3A3
:1083BA00A3A374BFF08B828A83A3A3E054EFF08B4C
:1083CA00828A83A3A3A3E561F0AE02AF038F828EF4
:0483DA0083A3E9F0A0
:0183DE00227C
:0483DF008F618D62BB
:1083E300E4F567743F2FF876087F807E257D007C57
:1083F30000AB66AA65A964A863D312A3B340267F22
:10840300007E967D007C00A863D312A3B3500C7545
:108413006740743F2561F87610800A756780743F62
:108423002561F87638E56745624401FFE56175F03B
:0D84330008A42402F582E43420F583EFF064
:018440002219
:108441008F828E83E014F557C3940440037FFF228B
:10845100E55775F008A42400F582E43420AF82F5D5
:10846100588F59E55725E024C6F582E4347FF5831A
:10847100E020E10FE55725E024C7F582E4347FF5DC
:1084810083E4F074232557F8E4F6E5592404F582D2
:10849100E43558F583E04403F0E55775F00DA42465
:1084A10002F582E43403F583E0FCA3E0FDA3E0FEE2
:1084B100A3E0F5668E658D648C637D06AF571283EC
:1084C100DFAF577D0112835A855982855883A3A353
